:1000000010C0189518951895189518951895189565
:100010001895189518951895189518951895189578
:1000200018958FE58DBFC8E3E0E24E2E81E08EBFCC
:10003000D1E0F1E05F2EA89584B7082E877F84BFBA
:1000400088E1992781BD91BDEEEFF0E0A0E6B0E038
:1000500088278D933197E9F76624B89AC098C09A9B
:10006000E1E0F0E007D0C098E1E0F0E003D0F7CFA6
:10007000F894FFCF88EE93E00CD03197D9F708952C
:100080003197F1F70895689462F80895E89462F85A
:100090000895EF93FF93EE27E82BE92B31F0E0ED85
:1000A000F7E03197F1F70197D1F7FF91EF910895BC
:00000001FF
